:04000000803119280A
:10000800803120007F08F800911D10288B31C5230E
:100018008031200091111628141C16288B31DB23FF
:10002800200014107808FF0009008B31A52B200050
:1000380069084A3E8600013087000108203A031902
:100048009F28B0280730F0006908473E8600013035
:100058008700700881006908493E860001308700E2
:10006800013524009900080024001E1B8128200067
:100078006908223E8600013087006908203E840016
:100088000130850000080102031864286908223E2F
:1000980086000130870001086907F00070088600B3
:1000A800013087000108240099000130F000200089
:1000B8006908223E86000130870070088107080021
:1000C8006908473E8600013087008101810A2400C3
:1000D8001E152330F000200069084A3E86000130D2
:1000E8008700700881003030F0006908483E8600BB
:1000F8000130870070088100080020006908473E29
:100108008600013087008101810A24001E152330F2
:10011800F000200069084A3E860001308700700818
:1001280081003130F0006908483E860001308700C0
:100138007008810008006908473E86000130870082
:100148000108013A0319DC2A043A03192628023A5D
:1001580003193828DC2A080069084A3E860001305D
:1001680087000108213A03196E2988290830F00010
:100178006908473E860001308700700881006908D9
:10018800493E8600013087000135F0007008F20012
:100198007214720824009900080024001E1BE1282C
:1001A8000330F00020006908473E860001308700D0
:1001B8007008810024009E15080020006908473E49
:1001C8008600013087008101810A24001E15233032
:1001D800F000200069084A3E860001308700700858
:1001E80081003330F0006908483E860001308700FE
:1001F80070088100080024001908F0002000690830
:10020800233E86000130870001086907F100710864
:10021800860001308700700881000130F00069080D
:10022800233E860001308700700881076908233E55
:100238008600013087006908203E8400013085006F
:1002480000080102031835290A30F0006908473E02
:100258008600013087007008810024009E121E1657
:1002680008000B30F00020006908473E8600013086
:1002780087007008810024009E161E1608000330AF
:10028800F00020006908473E8600013087007008AA
:10029800810024009E15080020006908473E86005A
:1002A800013087008101810A24001E152330F000E7
:1002B800200069084A3E86000130870070088100E6
:1002C8003230F0006908483E860001308700700827
:1002D800810008006908473E860001308700010850
:1002E800013A0319DC2A023A0319FF28063A0319CE
:1002F800BA280D3A0319D128023A03194329013AB9
:1003080003195029DC2A080069084A3E8600013092
:1003180087000108223A031D0800B92A0730F000B7
:100328006908473E86000130870070088100690827
:10033800493E8600013087000135240099000800F5
:1003480024001E1BBA292000690886000130870096
:100358000108240099000930F00020006908473E90
:1003680086000130870070088100080020006908B5
:10037800473E8600013087008101810A24001E154E
:100388002330F000200069084A3E860001308700CB
:10039800700881003130F0006908483E860001305D
:1003A800870070088100080024001E1BE7299E149E
:1003B8000630F00020006908473E860001308700BB
:1003C80070088100080020006908473E8600013057
:1003D80087008101810A24001E152330F0002000C7
:1003E80069084A3E86000130870070088100313074
:1003F800F0006908483E86000130870070088100D7
:1004080008000830F0006908473E86000130870080
:10041800700881006908493E86000130870001356F
:10042800F0007008F30073147308240099000800A2
:1004380024001E1B2C2A0330F00020006908473EC8
:100448008600013087007008810024009E1508008E
:1004580020006908473E8600013087008101810A33
:1004680024001E152330F000200069084A3E86004B
:1004780001308700700881003330F0006908483E79
:1004880086000130870070088100080024001908E0
:10049800F00020006908233E86000130870001082B
:1004A8006907F10071088600013087007008810033
:1004B8000130F0006908233E86000130870070088B
:1004C80081076908233E8600013087006908203EBD
:1004D800840001308500000801020318802A0A30D0
:1004E800F0006908473E86000130870070088100E7
:1004F80024009E121E1608000B30F0002000690828
:10050800473E8600013087007008810024009E164F
:100518001E1608000330F00020006908473E8600D8
:10052800013087007008810024009E150800200013
:100538006908473E8600013087008101810A24004E
:100548001E152330F000200069084A3E860001305D
:100558008700700881003230F0006908483E860044
:10056800013087007008810008006908473E86004E
:10057800013087000108013A0319DC2A023A0319FD
:100588004A2A063A03199229033A0319052A013A15
:100598000319A4290F3A03191C2A013A0319D82967
:1005A800033A03198E2A013A03199B2ADC2A080008
:1005B800080079084A3E860087010108203A031995
:1005C8004A2B5A2B0730F0007908473E86008701EE
:1005D800700881007908493E8600870101352400AA
:1005E800910008002400161B322B7908223E860051
:1005F80087017908203E840085010008010203185C
:100608001A2B7908223E8600870101087907F00035
:10061800700886008701010891000130F000790810
:10062800223E860087017008810708007908473E46
:10063800860087018101810A16152330F0007908A8
:100648004A3E86008701700881003030F000790842
:10065800483E860087017008810008007908473EF7
:10066800860087018101810A16152330F000790878
:100678004A3E86008701700881003130F000790811
:10068800483E860087017008810008007908473EC7
:10069800860087010108013A0319332D043A03192A
:1006A800E62A023A0319F62A332D080079084A3E49
:1006B800860087010108213A0319FA2B132C083008
:1006C800F0007908473E86008701700881007908A4
:1006D800493E860087010135F0007008F200721467
:1006E80072082400910008002400161B852B033093
:1006F800F0007908473E860087017008810096154A
:1007080008007908473E860087018101810A16158D
:100718002330F00079084A3E86008701700881007E
:100728003330F0007908483E860087017008810060
:10073800080024001108F0007908233E860087018C
:1007480001087907F10071088600870170088100A7
:100758000130F0007908233E860087017008810780
:100768007908233E860087017908203E84008501A8
:10077800000801020318CB2B0A30F0007908473E25
:1007880086008701700881009612161608000B3043
:10079800F0007908473E86008701700881009616A8
:1007A800161608000330F0007908473E86008701D6
:1007B800700881002400961508007908473E8600D5
:1007C80087018101810A240016152330F000790879
:1007D8004A3E86008701700881003230F0007908AF
:1007E800483E860087017008810008007908473E66
:1007F800860087010108013A0319332D023A0319CB
:100808009D2B063A0319632B0D3A0319782B023AEC
:100818000319D62B013A0319E12B332D0800790867
:100828004A3E860087010108223A031D0800112D5F
:100838000730F0007908473E86008701700881007C
:100848007908493E86008701013524009100080097
:100858002400161B3D2C79088600870101089100A9
:100868000930F0007908473E86008701700881004A
:1008780008007908473E860087018101810A16151C
:100888002330F00079084A3E86008701700881000D
:100898003130F0007908483E8600870170088100F1
:1008A80008002400161B622C96140630F000790804
:1008B800473E860087017008810008007908473E96
:1008C800860087018101810A16152330F000790816
:1008D8004A3E86008701700881003130F0007908AF
:1008E800483E860087017008810008000830F00043
:1008F8007908473E86008701700881007908493EDB
:10090800860087010135F0007008F300731473083E
:100918002400910008002400161B9C2C0330F000D2
:100928007908473E860087017008810096150800FF
:100938007908473E860087018101810A1615233010
:10094800F00079084A3E860087017008810033303C
:10095800F0007908483E8600870170088100080089
:1009680024001108F0007908233E86008701010859
:100978007907F1007108860087017008810001304D
:10098800F0007908233E86008701700881077908FE
:10099800233E860087017908203E840085010008EF
:1009A80001020318E22C0A30F0007908473E86005D
:1009B8008701700881009612161608000B30F000A7
:1009C8007908473E8600870170088100961616163A
:1009D80008000330F0007908473E86008701700858
:1009E80081002400961508007908473E8600870193
:1009F8008101810A240016152330F00079084A3E47
:100A080086008701700881003230F0007908483E7E
:100A1800860087017008810008007908473E860033
:100A280087010108013A0319332D023A0319B42C3E
:100A3800063A03191C2C033A03197A2C013A0319B4
:100A48002C2C0F3A03198F2C013A0319552C033A11
:100A58000319ED2C013A0319F82C332D080008006E
:100A6800F701F501F40124001D1F4E2D1D13200070
:100A78006908473E8600013087008101810AF40138
:100A8800F40A3630F2006908483E860001308700D3
:100A98007208810024001C1C572D1908F2007208E6
:100AA800F600F701F70AF4080319BE2ED22E240027
:100AB8009C1DD22E20006908213E86000130870047
:100AC80081010230F200782D24001C1E6D2D2000BB
:100AD8004C2E77080319D22E24009C1AAC2E1C1910
:100AE8007B2D0330F20020006908473EB82E043001
:100AF800F20020006908473E86000130870072082E
:100B0800810069084C3E8600013087008108031D7A
:100B1800B42D69084B3E86000130870001088B31EF
:100B28009B238531003A0319B22D20006908243E21
:100B38008600013087000108240099002000690818
:100B4800453E8600013087008101810A69084C3ED4
:100B58008600013087008101810ADC2D2000DF2D0D
:100B68006908453E8600013087006908443E8400D4
:100B780001308500000801020318DF2D6908453E91
:100B88008600013087000108243E6907F2007208D8
:100B98008600013087000108240099000130F20026
:100BA80020006908453E86000130870072088107E9
:100BB800F501F50AD22E69084C3E860001308700FF
:100BC80081014C2E24001C1E542E770803193D2E3B
:100BD8009C1E2C2E7608F20020006908233E860011
:100BE8000130870001086907F300730886000130A7
:100BF8008700720881006908233E8600013087005B
:100C080001081F3A031D0F2E6908233E8600013094
:100C180087008101182E0130F2006908233E860002
:100C280001308700720881070130F2006908213E0F
:100C3800860001308700720881077608F20069088B
:100C48004B3E860001308700720881003430352E13
:100C580020006908473E8600013087008101810A2B
:100C68003730F2006908483E860001308700720874
:100C7800810020006908213E8600013087000108B4
:100C8800F2006908203E860001308700720881075B
:100C98006908473E8600013087008101810AD22E0B
:100CA80077080319D22E24009C1E982E7608F2008D
:100CB80020006908233E8600013087000108690783
:100CC800F300730886000130870072088100690804
:100CD800233E86000130870001081F3A031D7B2E42
:100CE8006908233E8600013087008101842E013087
:100CF800F2006908233E86000130870072088107E8
:100D08000130F2006908213E860001308700720830
:100D180081077608F20069084B3E8600013087009B
:100D2800720881003430B52E1C1DAC2E20006908D5
:100D3800213E8600013087000108F2006908203E44
:100D4800860001308700720881070430F2007E2D8A
:100D580020006908473E8600013087008101810A2A
:100D68003730F2006908483E860001308700720873
:100D78008100D22E20006908473E86000130870096
:100D88000108013A03195B2D033A0319682D013A4A
:100D98000319E62D073A0319852DD22EF7080319F2
:100DA80075080319080024001D1A08001D160800FC
:100DB800210099171908873970389900FC3099056E
:100DC8008B31F52386318C31A72486312000C3006E
:100DD8004308D400A0308D319E2586312000540868
:100DE8008C310F24863120308E313F2686310030F9
:100DF8008C312B2486318731FE2786318731FB27BA
:100E080086318D31122586315730860000308700B3
:100E180044308400003085001030FF0016001A00AE
:100E2800FF0B122F443087314D2786318C314D24EA
:100E380086318C31762486312000C3004308D500E2
:100E4800D601083056020318482F5508C300560A21
:100E58002E2FC336890B2D2F431C382F5608443E9E
:100E6800860087018101402F1030C3005608443E98
:100E780086008701430881000130C3004308D60774
:100E880008305602031C292F443087314D278631FC
:100E98001D2F2000BB008230A900A7002708A90049
:100EA8003B08860087010108A7002708AA003B081D
:100EB80086008701413FAB003B0886008701423F1F
:100EC800AC003B0886008701433FAD003B08860025
:100ED8008701443FAE003B0886008701453FAF00CD
:100EE8003B0886008701463FB0003B088600870123
:100EF800473FB1003B0886008701483FB2003B08E6
:100F080086008701493FB3003B08860087014A3FB6
:100F1800B4003B08860087014B3FB5003B088600BC
:100F280087014C3FB6003B08860087014D3FB7005C
:100F38003B08860087014E3FB8003B0886008701C2
:100F48004F3FB9001130A7002708A0002930A8009A
:100F58002808A10060308D31EC2587318731BD2705
:100F680087312000A7002708BA003A08031D0800A7
:100F7800B22F20006908463E86000130870001082C
:100F8800113A031DE12F69084A3E860001308700A7
:100F98000108233A031DD82F6908203E8600013036
:100FA80087008108031DDA2F003008006908483ED1
:100FB800860001308700010808006908473E86005E
:100FC800013087000108013A031DF22F6908203E0D
:100FD8008600013087008108031DF42F00300800C7
:100FE8006908483E860001308700010808000B1791
:060FF8008B170800080041
:10171600FE0012001E00FE0B8C2B0034F000F101BF
:10172600640070080A3A0319992B992B710808006E
:10173600F000F101640070080A3A0319A32BA32BE9
:1017460071080800B33084008B308500573086005E
:101756000030870012308B318B2320008631DC2E3F
:1017660000340034003400340034003400340034D3
:101776001034103410341034103410341034103443
:10178600093400347908463E860087010108113A7B
:10179600031DD02B8231DD2208007908463E8600E3
:1017A60087010108103A031D08008E319A260800A9
:1017B60020006908463E8600013087000108113A7C
:1017C600031DE82B80311B20080020006908463ED7
:1017D6008600013087000108103A031D0800853194
:1017E6003425080023008C018D018E0121009513FC
:1017F6008C160C160C158E160E120E148E140E1553
:101806008E1524000E148E140E158E1521000D173C
:101816000D168D178D1608002000A1001030A000AF
:101826007908463E860087012008810021000D17B1
:101836000D16200021352400920094019501960191
:101846001508F0390E3895009417161495160800E9
:101856002000A1001130A0006908463E8600013034
:1018660087002008810021008D178D1624009C0119
:101876009D019E011D08F03908389D002000A10831
:10188600031D472C1330482C4F3024009A009C1718
:101896009D1608002000A901FF30A7002708AA000E
:1018A600FF30A7002708AB00AC01AD01AE01AF01C8
:1018B600FF30A7002708B0000830A7002708A000BF
:1018C6002930A8002808A10020308D31EC258C3164
:1018D6008731BD278C312000A7002708B1003108C9
:1018E600031D08006B2C20006808A901A9076708DA
:1018F600A801A807A001A00A2830A7002708A10070
:1019060020308D31EC258C318731BD278C3120007C
:10191600A7002708AA002A080319872CA001A00AF5
:1019260020308C31DA248C318731BD278C31200070
:10193600A7002708AA002A080319972C28308D31FA
:1019460058252000280808002000A30122000E0CBC
:101956002000A000A00C200C0139A1000230A13506
:10196600FF3E031DB22C2135A2002208A30422004B
:101976000E0C890C01392000A0000130A035FF3E75
:10198600031DC12C2035A1002108A30422000E0C42
:10199600013909072000A0002008A30422000E0830
:1019A60001392000A0002008A30423080800200015
:1019B600A200A008031908002008A1006908203E1B
:1019C600860001308700210881002208A1006908ED
:1019D600493E860001308700210881006908223EC1
:1019E60086000130870081016908233E86000130A8
:1019F600870081010530A1006908473E8600013055
:101A06008700210881002130A10069084A3E86002E
:101A1600013087002108810024001E140800803050
:101A26002000A7002708A9008030A7002708AA00E1
:101A3600AB01AC01AD01AE01AF01B001B101B20124
:101A4600B301B401B501B601B701B801B901BA01D4
:101A5600BB01FF30A7002708BC00BD01FF30A7006F
:101A66002708BE00FF30A7002708BF00FF30A700E9
:101A76002708C000FF30A7002708C1001930A700BB
:101A86002708A0002930A8002808A10060308D3161
:101A9600EC258D318731BD278D312000A700270821
:101AA600C2004208031D08004D2D2000A300A4011A
:101AB6006908203E86000130870081080319080066
:101AC6006908223E86000130870001086907A000E8
:101AD60020088600013087000108A100240823079A
:101AE600A200220886008701210881000130A0009B
:101AF6002008A4076908223E8600013087000108F5
:101B06001F3A031D8D2D6908223E8600013087008D
:101B16008101962D0130A0006908223E8600013021
:101B26008700200881076908203E8600013087006B
:101B3600013081025B2D2000A1002108A0002008B1
:101B4600F9007908203E8600870181017908213E47
:101B56008600870181017908223E8600870181017E
:101B66007908233E8600870181017908453E860073
:101B7600870181017908443E860087018101790841
:101B8600463E8600870181017908473E8600870127
:101B96008101810A7908483E86008701810179081A
:101BA6004B3E86008701810179084C3E86008701FD
:101BB60081017908493E8600870181012330A00012
:101BC60079084A3E86008701200881002100911588
:101BD60008002000A500A00803190800A601200897
:101BE600260203180C2E26082107A20022088600CA
:101BF60087010108A30026086907A40024088600B7
:101C060001308700230881000130A2002208A607C0
:101C1600F22D2008A2006908203E860001308700C8
:101C2600220881002508A2006908493E8600013085
:101C36008700220881006908223E8600013087005D
:101C460081016908233E8600013087008101053045
:101C5600A2006908473E86000130870022088100FD
:101C66002030A20069084A3E86000130870022081B
:101C7600810024001E1408002000A1002108A000F5
:101C86002008E9006908203E8600013087008101AE
:101C96006908213E86000130870081016908223EDD
:101CA60086000130870081016908233E86000130E5
:101CB600870081016908453E860001308700810161
:101CC6006908443E86000130870081016908463E66
:101CD60086000130870081016908473E8600013091
:101CE60087008101810A6908483E86000130870025
:101CF600810169084B3E8600013087008101690831
:101D06004C3E86000130870081016908493E860005
:101D16000130870081012330A00069084A3E860011
:101D26000130870020088100210014140800F70103
:101D3600F501F4012400151FB12E15137908473E4D
:101D4600860087018101810AF401F40A3630F20027
:101D56007908483E8600870172088100141CB92E56
:101D66001108F2007208F600F701F70AF4080319E1
:101D7600E42FF62F941DF62F7908213E8600870161
:101D860081010230D02E141A7C2F77080319F62F02
:101D9600941AD52F1419CC2F0330F2007908473E38
:101DA600DF2F79084C3E860087018108031DFA2E35
:101DB60079084B3E8600870101088B3191238E31CD
:101DC600003A03191F2F7908243E8600870101086F
:101DD600240091007908453E860087018101810A29
:101DE60079084C3E860087018101810A1C2F7908FB
:101DF600453E860087017908443E84008501000837
:101E0600010203181F2F7908453E86008701010845
:101E1600243E7907F2007208860087010108240033
:101E260091000130F2007908453E8600870172086C
:101E36008107F501F50AF62F79084C3E86008701E1
:101E460081017C2F141E832F77080319702F941E8F
:101E5600622F7608F2007908233E86008701010882
:101E66007907F300730886008701720881007908F4
:101E7600233E8600870101081F3A031D482F790873
:101E8600233E860087018101502F0130F200790838
:101E9600233E86008701720881070130F200790827
:101EA600213E86008701720881077608F2007908CC
:101EB6004B3E86008701720881003430692F79080D
:101EC600473E860087018101810A3730F200790892
:101ED600483E86008701720881007908213E860007
:101EE60087010108F2007908203E86008701720802
:101EF60081077908473E860087018101810AF62F0E
:101F060077080319F62F941EBE2F7608F20079087B
:101F1600233E8600870101087907F30073088600CF
:101F26008701720881007908233E8600870101082F
:101F36001F3A031DA42F7908233E860087018101DD
:101F4600AC2F0130F2007908233E86008701720823
:101F560081070130F2007908213E86008701720868
:101F660081077608F20079084B3E860087017208E1
:101F760081003430DC2F141DD52F7908213E8600D0
:101F860087010108F2007908203E86008701720861
:101F960081070430F2007908473E860087017208FF
:101FA6008100D42E7908473E860087018101810A87
:101FB6003730F2007908483E8600870172088100B2
:101FC600F62F7908473E860087010108013A031972
:101FD600BD2E033A0319C62E013A0319252F073AD7
:101FE6000319D42EF62FF7080319750803190800EC
:0A1FF6002400151A08001516080053
:020000040001F9
:04000E00E4FFFFDF2D
:00000001FF
